:020000041000EA
:1000000000B5324B212058609868022188439860DF
:10001000D860186158612E4B002199600221596106
:100020000121F02299502B49196001219960352056
:1000300000F044F80222904214D00621196600F024
:1000400034F8196E01211966002018661A6600F04E
:100050002CF8196E196E196E052000F02FF8012189
:100060000842F9D1002199601B49196000215960AB
:100070001A491B48016001219960EB211966A021F2
:10008000196600F012F800219960164914480160C1
:100090000121996001BC002800D000471248134993
:1000A000086003C880F30888084703B5996A0420EC
:1000B0000142FBD001200142F8D103BD02B5186610
:1000C0001866FFF7F2FF186E186E02BD00000240BE
:1000D000000000180000070000035F00212200005C
:1000E000F4000018222000A00001001008ED00E03C
:1000F00000000000000000000000000074B24E7A12
:1001000000200420F7010010CB010010CD010010E9
:10011000C9010010C9010010C9010010C901001077
:10012000C9010010C9010010C9010010CF01001061
:10013000C9010010C9010010D1010010D301001045
:10014000C1010010C1010010C1010010C101001067
:10015000C1010010C1010010C1010010C101001057
:10016000C1010010C1010010C1010010C101001047
:10017000C1010010C1010010C1010010C101001037
:10018000C1010010C1010010C1010010C101001027
:10019000C1010010C1010010C1010010C101001017
:1001A000C1010010C1010010C1010010C101001007
:1001B000C1010010C1010010C1010010C1010010F7
:1001C000EFF30580103800BE00BE00BE00BE00BECA
:1001D00000BE00BEF2EB887184390010A439001013
:1001E0003802001090A31AE71E481F49086006C88D
:1001F00081F3088810471D480068002801D019487D
:10020000F3E70DA40ECC002902D000F012F8F9E7B4
:100210001749184A002000E001C19142FCD116495B
:100220008847164988471649884700BEFDE701C937
:1002300001C29A42FBD37047A4390010C0000020CD
:10024000281000200C4900100000042000000420A9
:100250000C490010001004200010042000000000D1
:10026000704700000000000008ED00E0000000D032
:1002700028100020281B0020991C0010D502001017
:10028000911C0010F8B5C04606480749091A8B10A2
:10029000C90FC91810B5491003D0044B002B00D06A
:1002A000984710BD281000202810002000000000F2
:1002B000054B10B5002B03D00449054800E000BFF2
:1002C000FFF7E2FF10BDC04600000000E81A002062
:1002D000AC36001070B582B003F00CF9002100209C
:1002E00002F0A2FF01F02AFE1F211A2000F0A0F860
:1002F000002200211A2000F0B5F800211A2000F099
:10030000C5F8E02200261F4BD2011B6801AD134047
:100310001D4A136001200021404202F047F800F01E
:10032000B5FE002920D0FA220023920001F0B6F990
:100330000400831B0A2BEDD9002002F0B5FD002834
:10034000E8D004228021114B49001A600D4A13683D
:100350000B42FCD0536800212B802A00022300208E
:1003600002F0BEFD2600D5E7FA21890001F058F918
:100370000400831B0A2BCDD9002002F095FD002834
:10038000C8D0DEE700C0044000D0044000E00440D4
:100390007047C0467047C0467047C0467047C04669
:1003A000002070477047C04600487047143800105E
:1003B00000487047FC37001000487047D8370010DD
:1003C00070B5002822D0032829D8164B8000C558C4
:1003D000280003F0BFF8C0B2041C1F2814D8C026A0
:1003E000E4B2631CDBB25B00B6001E43002808D0F9
:1003F00000230D4AE95C01331180D9B202328C42EC
:10040000F8D80A48068070BD1F24E8E7C126054BCE
:1004100002220548196801F013FCB600F1E700203C
:10042000F1E7C046600F00200214002000140020F5
:10043000094A83009A1810B514684022544080324B
:100440002240064CC000A44663441A60044B9C46FC
:100450006044416010BDC04604C0014004D001406A
:1004600000400140074B8000C3181B68C900920080
:100470000A435A400C231340034A944660440360E5
:100480007047C04604C0014004D0014080000029EC
:1004900005D0064B9C464023604403607047044BE4
:1004A0009C46402360440360F8E7C04604E00140F6
:1004B00004F001400123D02283401206936293612D
:1004C000094A83009A1811684022514080320A403C
:1004D0000649C0008C4663441A60054B9C460523C0
:1004E000604443607047C04604C0014004D00140EE
:1004F000004001408023DB051868000F7047C046AC
:100500000FB400B5084883B001F0FAFC049B002B3F
:1005100007D005A91800019101F0A0FB034801F0E4
:10052000EFFC012001F0B2FBD0360010E0360010E5
:1005300070B5EFF3108C72B60D4D2B68002BFCD00C
:10054000BFF35F8F0724CB08C618C05C01230C40A3
:10055000A3401C000440034207D118433070BFF38E
:100560005F8F2C608CF3108870BD1000FFF7C8FF00
:100570002C0100D0F8B54746CE46884680B5EFF34B
:10058000108C72B6214D2C68002CFCD0BFF35F8F0D
:100590009A422CD8D4080727055D06190124174074
:1005A000BC402C421FD007210127894609E0D4080E
:1005B000055D06194C4639001440A1400C00294243
:1005C00011D001329342F2D201204042BFF35F8F3B
:1005D00000220E4B1A608CF3108800280FDBC0BC81
:1005E000B946B046F8BD254310003570EEE7BFF3BD
:1005F0005F8F00232B608CF310880120404243461C
:10060000002BECD00898FFF77BFFC0462C0100D0F0
:10061000044A1078431CDBB2172B00D91023137047
:100620007047C046700F002010B5064B064C82B0D4
:100630000100009318221F232000FFF79BFF02B048
:1006400010BDC046E4360010A41600200021044B63
:10065000044ABFF35F8F02C39342FAD17047C0468A
:10066000000100D0800100D0054B064A1360064A05
:10067000136053609360D36013615361936170475B
:100680008080808000E400E004E400E01F23184044
:100690001E3B8340002905D0C021044A4900535025
:1006A00013607047802201498B50FAE700E100E0B7
:1006B00070B50D00EFF3108672B60F4A1368002B69
:1006C000FCD0BFF35F8F0D4B10309B6884001B592B
:1006D0000B4A934203D09D4201D000F077FE074BB6
:1006E0009B681D51BFF35F8FBFF35F8F0022024BEA
:1006F0001A6086F3108870BD240100D000ED00E080
:10070000C1010010F0B557464E46DE464546E0B5FD
:1007100085B0060000911700EFF3108B72B66A4A9D
:100720001368002BFCD0BFF35F8F0025674B5D572C
:100730009A46002D00DAA9E06B00654C01935B1925
:100740009B009846A146C1444B4652469B791036C1
:100750001370604BB6009B6899590B1B2F2B33D934
:100760005D4B994200D0ACE0019B42469C465B4BFE
:100770006544AD0063535A4B0232A218043B9B1AE6
:100780001B05584A5B0D651913436B80564B0121BD
:10079000AB80FF23AB71009BEF71AB604B460B430B
:1007A00019004C4B9B689951BFF35F8FBFF35F8F6C
:1007B0000022454B1A608BF3108805B0F0BCBB4695
:1007C000B246A946A046F0BD01200A008243D37973
:1007D0008C46BB4231D84546130044491B1B5B4144
:1007E0005943090D3D4B63533D4B02356519043B9D
:1007F0005B1B1B053B4D5B0D2B43AA464D466B8097
:100800000425AC465546E044131F44441B1B1B05FE
:100810005B0D1D434B46997100999D809960494637
:10082000DF71334B01431360BBE75800C0188000F1
:100830002018C179B9422FD902000623D356002BC4
:10084000F3DA02932B4B61460393131D9A4604235C
:100850005B429C46E14450464B461B1A1B055B0D10
:100860009C46204B957198466346404603439380CF
:10087000019B5A199200039BA418A380029B1C4A57
:10088000A371009B2260E771A3608AE700F09EFDE0
:10089000002553465D574FE7908802934005131D8E
:1008A0009A46031561469C464046D444634604304C
:1008B0002018181AE0230005400D1B02184303906E
:1008C000C5E700F083FD4FE7240100D0241B002082
:1008D000740F002000ED00E0C101001000A1FFFF37
:1008E000A40F002000E0FFFF01BDFFFFAAAA000047
:1008F0000148804701BD000070B501240443EFF3B7
:100900000581EFF3108C72B6214A1368002BFCD0DE
:10091000BFF35F8F1F4B05001F4AED1A6D416A43FD
:10092000120D1E4D8900AE6852B27658A6421CD0F8
:100930000621595691421CD012215956914222D07B
:100940001E215956914220D02A2159560324914202
:1009500010D0134B19781A708171BFF35F8F00228A
:100960000B4B1A608CF3108870BDAB680D4C5C505B
:10097000EFE700246100091989005B18FF219971D4
:1009800009499980E5E70124F4E70224F2E7C0462B
:10099000240100D0740F0020AAAA000000ED00E09E
:1009A000241B0020C101001001BDFFFF024B9C462B
:1009B00061448900016070474000003470B5114CFB
:1009C000114DAC420FD2FF262368002B0CD0FFF74D
:1009D0001FFE01002000FFF7E9FFA680BFF35F8F35
:1009E0000834AC42F0D370BDFFF712FE01002000C6
:1009F000FFF7DCFF2671BFF35F8F0834AC42E3D30F
:100A0000F1E7C046201000202810002010B5040097
:100A1000FFF7FEFD01002000FFF7C8FFFF23237151
:100A2000BFF35F8F10BDC04610B504000120FFF773
:100A3000FBFD034BC3189B002360BFF35F8F10BD0A
:100A4000400000340A4B1968EFF3108072B60A6850
:100A5000002AFCD0BFF35F8F1B68BFF35F8F0022BB
:100A60001A6080F3108840BF002000217047C04604
:100A70001C1B0020F0B5DE4657464E464546E0B505
:100A800083B0EFF3058203231340B54A990052580F
:100A90000091904601229A409346B24B1A60B24BA5
:100AA00001935B46B1484363434608229B5E9946E7
:100AB000002B3ADA43469B881BB2002B00DB9DE0FB
:100AC00043469B79002B00D0E1E0434608241C5F9D
:100AD000002C20DB43465A6963001B19DB00D31846
:100AE0009D68DC686B1C00D103E1A0480099844636
:100AF0006144826A0B69AE1A9B1A9E4213D35A460E
:100B0000036A1A420FD0994800F0B8FA8C4202DC0E
:100B1000C7D18542C5D940BF03B0F0BCBB46B24681
:100B2000A946A046F0BD0D61EDE7424652695B0063
:100B300092464B44DB009A4453469E68DF6800F0BF
:100B40009DFA8F42B6DC00D1F8E0002F00DAD9E040
:100B50005246534654691B69019A934200D1CCE036
:100B6000414652460820085E528800042100104386
:100B7000984704000D0023002B4300D1C2E0002D54
:100B800000DBDFE030003900001BA94153469860CC
:100B9000D96000229A5E002A00DA8BE743465D693D
:100BA00053009C18E4002C19A768E4688C4200DD0F
:100BB00080E702D1874200D97CE746463281083679
:100BC0000DE08C4200D1C6E01E000023F25E002A38
:100BD0000ADB53009C18E4002C19A768E4689B18F2
:100BE000DB00EB188C42ECDD53461A804B46338019
:100BF00043469B881BB2002B00DA61E743461A6923
:100C0000EFF3108172B61368002BFCD0BFF35F8F37
:100C100043469E88012342465B42938036B2136965
:100C2000BFF35F8F00221A6081F31088002E00DA74
:100C300046E743465D69083342469C467700BF1944
:100C4000FF00EF19BB68604698460823D15E9246C4
:100C5000FC68002907DA0EE0A24246D01800002303
:100C6000C15E002906DB4B005B18DB00EB18DA687D
:100C7000A242F1DD524606800023FE5E3980002E3E
:100C8000DCDA904643469B79002B00D11DE7002318
:100C900042469371434646460821595E08364B1C2E
:100CA00000D138E747468946556902E006004B1CEB
:100CB00018D04B005B18DB00E8180A008C46E95E90
:100CC00043881BB2002BF1DA01235B42DC178360FF
:100CD000C4604A4503D031803B8903803A81E146B4
:100CE0004B1CE6D1B8464C46F2E69A684245B5D967
:100CF000C0E7631C00D0F8E605E7200023699847A9
:100D0000002825D1534642461B8813811269EFF310
:100D1000108372B611680029FCD0BFF35F8F424682
:100D2000514652880A804246494651801269BFF3B3
:100D30005F8F0021116083F31088BBE6864200D8E4
:100D400003E7B7E6094800F099F9001969411DE782
:100D5000656824680FE7874200D835E744E7C04656
:100D6000001B00203C700540750A00100040054043
:100D700070B52E4C2569002D04D00A212C48FFF7B0
:100D800015FE70BD2B4E0321300000F06DF9E660BA
:100D9000FFF73EFC284B03229C46D02322701B0603
:100DA0001B6801216370254B6044A3600F23800002
:100DB00020610220638063694942A1801980023169
:100DC000198647311D83585218315A5275325C3991
:100DD0009952183201319952183201319952183210
:100DE00001319952083518329D5202311832995208
:100DF00018320131995218320131995218320131A9
:100E000099521832013199521832013199520C4BD2
:100E10000C49DC6001303562FFF74AFC01210320F8
:100E2000FFF734FC084B1D60A7E7C046BC0F00204D
:100E30001C1B00200040054040000034FFFF100054
:100E4000001B0020750A00103860054070B50100D5
:100E50000469EFF3108C72B620680028FCD0BFF351
:100E60005F8F02200D5E4C6968004019C000241895
:100E7000002D37DB208848800869BFF35F8F00268C
:100E800006608CF31088E360638804980133206166
:100E90005B0405985B0CA26060611A1C002B1FD0DC
:100EA00093B22804628018430A69EFF3108C72B67B
:100EB0001368002BFCD0BFF35F8F8B8823808D805D
:100EC0000B69BFF35F8F00221A608CF310880B78D8
:100ED00001329A40CB6808498C4663441A6070BD61
:100EE0000122DDE70B69BFF35F8F00221A608CF3EC
:100EF000108801204042F2E73C20000010B54389F1
:100F00000A1493421ADD53009B184269DB00D31880
:100F10000469EFF3108C72B62268002AFCD0BFF38C
:100F20005F8F5A88090494B2090C8A4208D0036979
:100F3000BFF35F8F00221A608CF31088002010BD71
:100F40008022120214435C80012302698371BFF383
:100F50005F8F002111608CF31088044902788C4661
:100F60009340C268012062441360E8E73C2000001F
:100F7000F0B5D6464F464646C0B504000D0082B0D7
:100F8000EFF305878946002F0ED0344900204B6AC5
:100F9000AB4203D38A6A0130A24226D302B0E0BC3E
:100FA000BA46B146A846F0BD2D4B9846DB689A4636
:100FB000434650461E7800F061F80B00514602008F
:100FC0000436B600715820008E1A2900801A994103
:100FD0008F4211DC0ED020BF204A0020536A4B45BF
:100FE000DCD3926A0130A242D8D25B1B5A1E9341D5
:100FF000D8B2D3E78642EED900F048F822002B00A1
:10100000121A8B41002B1ADB00230193154B22008F
:10101000009340462B00FFF719FF011E0FDD0F4B19
:101020005A6A4A4517D39B6AA34212D34046FFF738
:1010300065FF0A4A0020536A4B45AFD3D1E7074A00
:101040000020536A4B45A9D3926A0120A242A5D23F
:10105000CBE74A45EAD120BFE8E7C046004005405B
:10106000BC0F0020450A001010B5024A0248FFF7E5
:101070005FFA10BD00370010A81600200300416A77
:101080000A00986A596A8A42FAD17047034B596A32
:101090000A00986A596A9142FAD1704700400540A7
:1010A000F8B5DE464E4657464546E0B58B46050048
:1010B0000A991800160000F0B3FA0A9B6C001F0290
:1010C000324B64199C46A4006444636881469F4285
:1010D00000D967602B1FDBB29846012B30D9C023A3
:1010E00080229B01E31812011A60294BAD00595967
:1010F0009A4600291BD17301E026226853401E4006
:10110000802342465B01E3181E60012A30D9802308
:1011100080229B01E31812011A6053464A46676019
:101120005A51F0BCBB46B246A946A046F8BD586924
:1011300000F076FA013043001B18033BFDD2DAE7DA
:101140005B46012BCBD1C02303229B01E3181A601D
:10115000023AA3681A42FCD07301E0262268AD006F
:1011600053401E4080230A4A5B019246E3181E60EA
:101170005A462168514003220A401A6001225B4608
:101180009A40A3681A42FCD0C1E7C04600800040E4
:10119000AC160020F0B546464F46D646C0B51F00F7
:1011A000344B44009C462418A40064446368884679
:1011B0001600FF2B02D880235B006360031FDBB2A5
:1011C0009A46012B30D9C02380229B01E3181201DB
:1011D0001A60294B85005959994600291BD1730182
:1011E000E026226853401E40802352465B01E318EC
:1011F0001E60012A30D9802380229B01E31812014E
:101200001A6080235B0063604B465F51E0BCBA46C6
:10121000B146A846F0BD586900F002FA013043001B
:101220001B18033BFDD2DAE74346012BCBD1C02389
:1012300003229B01E3181A60023AA3681A42FCD009
:101240007301E0262268850053401E4080230A4A2D
:101250005B019146E3181E6042462168514003221B
:101260000A401A60012342469340A2681342FCD010
:10127000C1E7C04600800040AC160020014B800052
:10128000C0587047AC160020F8B5040021481E0075
:1012900017000D0000F0C4F90100380000F0C0F99B
:1012A000069B36041B031E432368002B20DB1A4BCE
:1012B0001A49E3185A1E93418022920194465B42D8
:1012C0001B0B174A1B0363441360164A13601F006D
:1012D0000A689743FBD1144B2560E2182123A060D4
:1012E00013602368002BFCDA0823E6601360F8BD66
:1012F0003F2322681340AB42D9D1A3681B051B0DC5
:101300008342D4D1EE22E368D2021340B342CED15D
:10131000EDE7C046001BB7000040FDBF08C000401D
:1013200000E0004000F00040043000008023024A4A
:101330009B000B43D362704700800540142310B517
:101340000100188804331B88984710BD162310B578
:101350000100188802331B88984710BDF8B547462E
:10136000CE4680B50F1E19D01423994604330400CD
:101370000025012698464B461888434621681B885D
:10138000984701C4431E9841013540420640AF4290
:10139000F1D13000C0BCB946B046F8BD0126F8E72F
:1013A000AA23064A1B0113608D235B00D360044906
:1013B000044B19605368002BFCDA70470040024070
:1013C00000B0FA00006002407047C04610B5014806
:1013D000FFF796F82437001070B5074D074EB54259
:1013E00009D20024013E761BB60808CD9847230099
:1013F0000134B342F9D170BD68360010A436001034
:10140000054B064A06491A60064A074B1A60100047
:101410000B689843FBD1704700E00040BFCDFBFE56
:1014200008C00040FE7F3C0000F00040044BDB6C35
:10143000002B03D18022034BD2021A607047C046B2
:10144000000011504C201150044A054B1A60054A07
:101450001368DB018033FBD17047C046FFFFFF01FB
:1014600000F0004008C000404022034B9A675A67D2
:101470001A67DA667047C04600F0014010B5FFF702
:10148000E5F810BDF8B52749274C284D641AA61079
:101490003200302E00D930222800920000F0D0FB1C
:1014A000BC2C3BD830202F232C196407204A801BEA
:1014B000E40F9B1B052B16D93700002C02D0B3007C
:1014C000771CEA50001B33199B004108EB18C90038
:1014D000C9181A605A6008339942FAD101230342AD
:1014E0001CD09843C619B300EA50731C2F2E15D098
:1014F0009B00EA50B31C2E2E10D09B00EA50F31C28
:101500002D2E0BD09B00EA50331D2C2E06D09B00B5
:10151000EA50731D2B2E01D09B00EA50054B9D60B5
:10152000F8BDC04600010010C001001000000020FE
:10153000C101001000ED00E0002310B5294C82B07D
:10154000A367FFF72DFF0122274B1A60636C012B65
:10155000FCD10322254B1A60224A936B012BFCD14C
:10156000013300930121224A22480433FFF78CFE05
:10157000052301210093204A2048FFF785FE002221
:10158000022104201E4BFFF705FE00220121052049
:101590001C4BFFF7FFFD0022002107201A4BFFF72D
:1015A000F9FD002200210820174BFFF7F3FD8023EF
:1015B000DB000093002200210920134BFFF770FD90
:1015C0000022104B00210620FFF7E4FD0420FFF766
:1015D00055FE0E4900F024F801000020FFF7A6FE9A
:1015E00002B010BD008000403CB0004030B0004070
:1015F000002F685900800240008C864700C00240DE
:10160000001BB70040597307006CDC0240420F001A
:1016100001480421014B1847E00F00205D13001022
:10162000114A936F9B0813D210665166002905D0AA
:10163000FFE7FFE7FFE7516F106F704704B5002821
:1016400001D00020C04301F0D7FF002104BDC046F7
:10165000F0B5146E556E576F166FFFF7E5FF146601
:10166000556657671667F0BD000000D094464A4A99
:10167000926F9208624601D228E0C046F0B5464E0D
:10168000346E756E776F366F00F020F89446424ADC
:1016900014665566576716676246F0BD94463E4A23
:1016A000926F9208624601D254E0C046F0B53A4EBD
:1016B000346E756E776F366F00F04CF89446364A8C
:1016C00014665566576716676246F0BD002B24DB2B
:1016D00011D000293EDA00B5C943404200D10131A2
:1016E00000F038F8C943404200D10131DB43524297
:1016F00000D1013300BD002AEBD1002801D100291F
:1017000005D00020C90FC90701D1C043410800B569
:1017100001F06AFF0022002300BD00B500290ADBAA
:10172000DB43524200D1013300F014F8C943404278
:1017300000D1013100BDC943404200D10131DB433A
:10174000524200D1013300F005F8DB43524200D190
:10175000013300BD002923D1002B18D1002A0CD061
:10176000BC460D4F38667A6600210023FFE7FFE78D
:10177000FFE77A6F386F67467047002801D0074847
:10178000010000B501F030FF0022002300BD02007F
:101790000B00002000217047000000D0FFFFFFFF7A
:1017A000002B00D0BFE0130C28D1002AE7D080B472
:1017B000114F39667A66FFE7FFE730B4040C7B6FA0
:1017C000396F1B0423433B667A66FFE7FFE7FFE7B9
:1017D000C04684B27B6F3D6F1B0423433B667A6631
:1017E000FFE7FFE7C04600232C042D0C7A6F386F0B
:1017F00000196941B0BC7047000000D0F0B59446B4
:101800000025140E01D112020835140F01D1120166
:101810000435940F01D192000235D40F01D152004A
:101820000135D40B0134254F7C66254C3C660E0CEB
:1018300093B2FFE7FFE7FFE73C6F6643360C7703A1
:10184000BE467343DF0B5B04C01AB941130C7343EC
:10185000DB18C91ACE086643360CB64493B27343FC
:101860001F0F1B01C01AB941130C73431F0B1B053B
:10187000C01AB941860D8F023E436643360C092DCE
:1018800024DB520A7243801A7703460A6643360CF9
:1018900016235B1BDE40DF40BF1964466643821B94
:1018A0007046043506330100D940A840C01900D362
:1018B0000131A24206D20023F0BD0000000000D09A
:1018C000FFFFFFFF121B0130F3D3F1E709277F1B56
:1018D000FE406446A2B27243801A00D20139220C43
:1018E0007243130C1204821A99410B00704604359E
:1018F00013370100F940A840801900D30131002BB3
:1019000002D1A2420AD2F0BD013000D30131121B34
:10191000FAD2013BF8D1A24200D2F0BD013000D38F
:101920000131121BF7E7F0B51C0C00D080E00CB4BD
:1019300000251C0A04D11B02160E3343120208357F
:101940001C0B04D11B01160F3343120104359C0BF1
:1019500004D19B00960F334392000235DC0B02D179
:1019600092185B4101351C00971864410134464FC1
:101970007C66464C3C660E0CFFE7FFE7FFE7C0467F
:101980003C6F6643360C7703BE4697B27743C01B65
:1019900000D20139C01B00D201399FB27743C91B65
:1019A000C91B170C77437E04FF0B801BB941CE087F
:1019B0006643360C0C2D33DBB644120B1F053A433D
:1019C0001B0B97B27743C01B00D201399FB27743FC
:1019D000C91B170C77433E043F0C801BB941860D91
:1019E0008F023E43664329277F1BFE400C3D77460E
:1019F000AF40BF1930BCA2B2ABB272437343801A7E
:101A00009941220C7243130C1204801A994102006E
:101A10000B000137001BA941F9D2781E0021F0BD4F
:101A20000C277F1BFE4077467F0BAF40FF19E0E796
:101A300000245D1C07D0144F7D663966FFE7FFE781
:101A4000FFE7FFE73C6F95B29EB265436643401BDC
:101A5000B141150C1E0C6543664336042F0C3E4302
:101A60002D04401BB141994204D202000B0020001A
:101A70000021F0BD01D19042F7D3801A9941013481
:101A80009942F2D3F6E70000000000D0FFFFFFFF0D
:101A9000132370B51D78012D19D014DD1F48FFF7F1
:101AA00055FC06001E48FFF751FC1E4C80223100F9
:101AB000200000F0C5F8022D2DD01B48FFF73EFC9A
:101AC0001A4B186070BD1A4B164CA364F5E7184BFF
:101AD000144C23606360A360E36023616361A361CE
:101AE000E36123626362A362E36223636363A363CC
:101AF000E36323646364A364E36423656365A365AC
:101B0000E36523666366A366E36623676367A3678B
:101B1000E367A364D1E7064BA364CEE75344000018
:101B200053460000A81100204C330000181B002071
:101B3000351B001007B5604601880A0A0230DF2A0B
:101B4000FAD1C9B2820804D3028840880004104345
:101B500000E00068014A5050039007BDA811002022
:101B600051434343C9188C46110C83B24B4310B404
:101B7000040C614392B280B2504362431C041B0CBC
:101B8000001910BC59411304120CC0185141614492
:101B900070470000132310B512481C78FFF7D6FBDE
:101BA0000100012C0AD003DD80220F4800F048F824
:101BB0000E48FFF7C3FB0E4B186010BD0A4C5422B1
:101BC000200000F03DF80B4B6365A365E3652366D9
:101BD0006366A366E36623676367A367E3672362BD
:101BE000E361E5E753460000A81200204C330000F3
:101BF000181B0020F91B001007B5604601880A0A6F
:101C00000230DF2AFAD1C9B2820804D302884088A0
:101C10000004104300E00068014A5050039007BDE3
:101C2000A812002001480421014B1847F00F0020A2
:101C30005D130010014B1B6818470000F00F0020D7
:101C4000014B5B6818470000F00F002010B500281A
:101C500000D110BD00F008F9FBE7C04610B5094AF5
:101C60000300146884B0002C08D0012200910648BB
:101C7000524203A9A047012004B010BD00F040F972
:101C80000020F9E7E01A00204D1C001000BEFDE71F
:101C900010B5FFF7FBFFC04670B5FFF79DFB074D82
:101CA000074EB54209D20024013E761BB60808CD86
:101CB000984723000134B342F9D170BDA436001017
:101CC000AC360010030010B5080011001B689847DF
:101CD00010BDC046F0B5C64600B5437D07000D00F7
:101CE0001600002B38D0002A2EDD00216A1E9046F7
:101CF0006A5C037D4C1C00200A2A0CD0A64216D038
:101D000043461B5D21000D3B5A4253416A5CDBB2E6
:101D10004C1C0A2AF2D1002BF0D1884217DB022199
:101D200010483B689847A64207D02000E8E7864263
:101D300003DD311A3B6828189847AD19013D2B780F
:101D40000D3B5A4253413B7580BCB846F0BD091A61
:101D50003B6828189847E2E7036811002800984775
:101D6000F2E7C0467C380010F0B5DE4657464E46D6
:101D70004546E0B585B017001C0006000D00FFF7D2
:101D800085F90023314A12184B41802109068B4204
:101D900002D301222E4B52422E4908008A4601F0FE
:101DA00043FC01906B1C03D1300001F0D3FB050014
:101DB000002C26D0284B9846284B1C68002C15D0A8
:101DC000002F21D1264F02E02469002C0ED0236879
:101DD000002BF9D03B68002B01D09C42F4D12000AD
:101DE0002A003100C0472469002CF0D1019B002B50
:101DF00028D1280005B0F0BCBB46B246A946A04693
:101E0000F0BD184B9846D7E7154B994602ABDF1D3E
:101E10000A239B4602E02469002CE7D02368002BAC
:101E2000F9D04B461B68002B01D0A342F3D12A0006
:101E300031002000C0475B460122390020003B7082
:101E4000C047E8E7504601F0C7FBD2E740420F0029
:101E5000FFFFFF7F20100020D51C0010D4160020AB
:101E6000DC160020C51C0010F0B5CE46474680B5F4
:101E700083B06B460600DD1D2870FFF707F90023CD
:101E80001A4A12184B41802109068B4202D30122C3
:101E9000174B524217490800884601F0C5FB164B04
:101EA00081461C68002C14D0144F02E02469002CD9
:101EB0000FD02368002BF9D03B68002B01D09C4247
:101EC000F4D1200001222900FFF704FF2469002C2F
:101ED000EFD14B46002B05D1300003B0C0BCB94652
:101EE000B046F0BD404601F077FBF5E740420F00F9
:101EF000FFFFFF7F20100020D4160020DC160020FA
:101F000070B5040001F026FB012301000500012249
:101F10002000FFF729FF084B1C68002C06D06368DF
:101F2000002B05D098472469002CF8D1280070BDFB
:101F30002469002CF3D1F9E7D416002001230121F4
:101F4000084A1360084A1360084A08001368984357
:101F5000FBD1074A11608021490013680B42FCD075
:101F60007047C04600E0004000F0004008C000405C
:101F700000C00440F8B500F043F90C23194DFF22CE
:101F8000AB6705201849FEF7BDFB184C4022002125
:101F90002000FFF74FFE4027002301262121144A8D
:101FA00066702783A260136063545F316184453992
:101FB0006354104A10496360E2602787A1620B6096
:101FC0006362E26201F0F8FA80239B052E64EB6401
:101FD00090230A4A0120EA508022094B5202DA6417
:101FE000F8BDC046000011501D030020E01600207F
:101FF00084001050000110508000105010D00100DB
:102000000020115010B501210520FEF73FFB10BD47
:1020100010B500220021024800F012F910BDC046A0
:1020200000170020044B1970002904D08021902350
:10203000024A8902D1507047211B00200020115014
:102040000B785B0602D14B78052B00D070478A785D
:10205000014B1A60FAE7C04600001150F0B5C646C1
:10206000C87800B58007830F1800012B60D08F78E7
:102070000A794B797F213940FC091B024E0013433A
:10208000334D32195201AA189770012767405770D3
:1020900000275B055B0DD7701383D076B846CA0066
:1020A000012C32D02B4FBC468F016244BC46AC445D
:1020B0006746BA6047461760002932D0264AC900F1
:1020C00090466246414451603F223F339343022889
:1020D00037D0224937190A687F01D3180B6020498D
:1020E000EF19FA608B422ED836197601AD19EB7EC6
:1020F0001C499B064A4013438022120613436A6818
:102100001360012080BCB846F0BD174FBC468F015C
:102110006244BC46AC446746BA6247461760002931
:1021200008D1002364012C196360104BE360E8E7D9
:102130000020E7E70B4AC9009046624641445162DD
:10214000C2E75B00C5E7FFF741F9FA68CCE7C04694
:10215000E01600208400105004001050E41A002003
:10216000FF0F105000001050800010500001105060
:1021700010B501F021FA10BD10B57F200C002040F1
:102180004000E409110000191A00034B4001C01877
:1021900000F056F8012010BDE01600207F23180043
:1021A00010B50840CA090B4203D107497D3B9B1A71
:1021B0008B66400080188022044B40010021C0182B
:1021C000120101F041FA10BD00201150E01600206C
:1021D0007F22130010B50B400A4200D110BDC9097F
:1021E0005B005B1804485B01C01800230022034910
:1021F000C37001F029FAF1E7E0160020FFF7FFFFB6
:1022000080220A4B520410B51A60094B09491A6022
:1022100010000B689843FBD1802200215201064830
:10222000FFF708FD0922054B5A6710BD00E000408A
:1022300000F0004008C000400000105000001150A5
:10224000002310B5C38201338282837601610400CA
:1022500001F0DAF9002804D080219023074A89028E
:10226000D150200001F0F8F9002802D00123237793
:1022700010BD200001F0E0F9FAE7C046002011503F
:10228000002070477047C0467047C0460020704726
:102290000020704700207047024B5878431E984139
:1022A000C0B2704788140020024B18784007C00F56
:1022B0007047C04688140020F0B5D6464F464646C3
:1022C000C0B52F4B07009A461B780E00FF2B01D09C
:1022D000012041E000293ED0002154222948FFF787
:1022E000A9FC0022284C294B20001A70FEF78EFB17
:1022F000274B1C60274C2000143CFEF795FB200068
:1023000001F0D8F8244B254D1C60254B002B28D01C
:10231000280000E000BF234B18602B78224A0024DD
:102320009146204A90460EE043461B6862019B1886
:10233000002B10D05B68002B0DD0984701342B7810
:10234000E4B2A3420FD3A342EED8E31A5B014B449D
:102350005B68002BF1D10020E0BCBA46B146A8462C
:10236000F0BD2B78DAE75346310038001F70FFF7D5
:1023700001FE0028EFD03800FFF744FE0120EBE714
:102380001C1000208814002080140020221B002034
:10239000DC14002014100020E0140020201B00207A
:1023A00000000000A813002028390010F0B5DE4618
:1023B00057464E464546E0B5CA4B8FB003931B784F
:1023C000FF2B00D146E1C84BC84E9B465F46C84B29
:1023D0000BAC0293C74B019335686A69EFF3108128
:1023E00072B61368002BFCD0BFF35F8FA961280081
:1023F000210000F0BDFF6A69AB69BFF35F8F002168
:10240000116083F31088002800D123E16378082B42
:10241000E2D89B00FB589F466368002BDCD0A06885
:102420009847D9E77F222179B14D0A405300EB1834
:102430009846C809804440460123303005799D43C1
:102440000571057903339D430571002A00D108E128
:102450004346A94A1B7D1278934200D3F8E0A74A6D
:102460005B011568ED18002D00D1F3E0A3686279D7
:102470002078AD69A847AFE7A14A1378002B00D1B7
:10248000E8E01378013BDBB213701378002BA3D183
:102490000122974D01212B78042013432B70342304
:1024A000EA5C8A43EA54EA5C8243EA540133EA5C18
:1024B0008A43EA54EA5C8243EA542378002098462F
:1024C00000F060FC602223791A40602A00D1F3E01A
:1024D000402A00D1F9E0DB06DB0E012B00D117E129
:1024E000022B00D1CCE0002B00D0E5E0202A00D167
:1024F0000FE2002A00D0DFE06379092B00D9DBE08E
:10250000804A9B00D3589F46794D2B78DB0700D437
:1025100062E7FDF743FF5FE7029BDB78DB0700D450
:102520005AE76068FFF7B0FE56E7714D2B78DB077E
:1025300000D451E728780007C00FFDF72DFF4BE7C7
:1025400023786C4A984693466B4B6C4A9946310007
:1025500092463A0046464F460025914688461B78EB
:102560000EE053461B686A019B18002B00D17EE0E9
:10257000DB683000984701353B78EDB2AB420CD3B5
:102580009D42EED3EB1A5B015B44DB683000984759
:1025900001353B78EDB2AB42F2D2554D54220021C9
:1025A0002800FFF747FB1022FF21281DFFF742FB01
:1025B00028002022FF21143046464F46FFF73AFB01
:1025C00000F0D6FB2379AB7006E723784B4A984698
:1025D000494B924699463200BB46464600254F4637
:1025E00090461B780DE053461B686A019B18002B30
:1025F00041D0DB683000984701353B78EDB2AB4203
:102600000ED3AB42EFD8019AEB1A94465B016344B8
:10261000DB683000984701353B78EDB2AB42F0D231
:10262000029D542200212800FFF704FB1022FF2105
:102630003548FFF7FFFA28002022FF2114304646D4
:102640005F46FFF7F7FA00F093FBFDF7A3FEC3E642
:10265000934213D00FB0F0BCBB46B246A946A04689
:10266000F0BDA3686279207800F0A0FBB4E646468E
:102670004F461F4DA4E746465F46E4E71D4DF5E68D
:102680007023217A0B4217D1C80983460F330B40C0
:102690005B0099461848EB185B441B7D0078834229
:1026A00061D216485B01006882469A44002A00D134
:1026B0004EE15346002B5ED120780021FFF76EFDDE
:1026C00080212078FFF76AFD86E6104800F05AFB6B
:1026D000012140460CAAFFF7D3FD002800D07BE67D
:1026E000EAE7C0461C10002080380010E0140020EB
:1026F0008814002028390010201B0020A813002077
:10270000221B0020A43800108C140020812200100D
:10271000237A0F2BD0D8D54AEB181B791278934225
:1027200034D3C9D1D24D686900F02CFB0121404659
:102730006B690CAA9847002800D04DE6602215006E
:1027400023791D401A42B7D163790A3B012BB3D8D4
:1027500000F018FB63790A2B00D17DE140460CA9FB
:1027600000F09AFA38E6834200D0ECE0C04B9A467B
:10277000002A00D1ECE05346586900F003FB5346B1
:10278000012140465B690CAA9847A6E7B94A5B015C
:102790001568ED18002DC6D18EE7A3799A466B789F
:1027A0009A45DBD06B78002B00D028E153466B7044
:1027B000002B00D120E150460138C0B2FDF7FCFDEE
:1027C000002800D171E14378022B00D06DE1012295
:1027D000C179A9468B11491113400A4030211201D9
:1027E0005B0113432A788A4313432B7009239B46CA
:1027F00083445D46B346C37882781B021343C318F3
:1028000006939A4B04970593994B0893994B9A46D4
:10281000994B0993069BAB4200D849E16B780122A2
:102820000B2B03D12B78EA78ED186B78042B00D0B2
:1028300038E1069B00265B1B9BB20793059B1700A4
:102840001B7818E053461B6872019B18002B00D1BF
:1028500028E1290040461B69079A9847082803D9B0
:10286000079B834200D30BE1059B01361B78F6B230
:10287000B34200D216E1B342E4D8089AF31A944660
:102880005B016344E5E76B780AAA023213704046A5
:1028900001230CA900F016FA9EE5E3881A0AD8B2C3
:1028A0000F2A00D908E775499300CB589F460CA81A
:1028B00000F06EFA4046A179FFF7AAFB02222B78BE
:1028C00013432B7088E5E388012B00D0F4E608223F
:1028D0002B78404693430CA92B7000F0DDF97BE583
:1028E000022029780AAB9A1C8B068908DB0F01406D
:1028F0000B431380404602230CA900F0E3F96BE57B
:10290000E388012B00D0D7E608222B7813432B70E5
:1029100024E7237A0F2B00D9CEE6544AEB181B7913
:102920001278934228D2534A5B011568ED18002DA6
:1029300000D1C1E6686900F025FA012140466B69C3
:102940000CAA9847C9E6002A00D0B5E600239A46AB
:1029500062790220130004928343012B11D0002AD4
:1029600000D0A9E62B004B445B4430331B790AAA04
:102970009B07DB0F0232BCE7934200D09CE63C4D44
:10298000D8E7E388002B12D1039B1878049B012B16
:1029900023D0FFF703FC4B460221EB185B44303396
:1029A0001A790A4301211A711A790A431A71534696
:1029B000002B00D110E5586900F0E4F953460121DD
:1029C0005B690CAA40469847002000F0DBF93523EC
:1029D000EB5CDB0700D5FFE4C0E6FFF7F9FB4B46F5
:1029E0000221EB185B4430331A798A431A711A7941
:1029F00004998A431A71DAE7FDF7CCFCAEE60021B0
:102A00004046FFF70FFB4046FFF7B2FB002293461C
:102A1000174AAB780592174A049306922A00134B83
:102A20005D46994693461B780EE0069B6A011B683B
:102A30009B18002B55D0DB68404698474B46013524
:102A40001B78EDB2AB4238D39D42EED3059AEB1A18
:102A500094465B016344EEE70AAB9A1C40460123AF
:102A60000CA9157000F02EF9B6E4C046201B00201A
:102A700028390010A81300209C140020CC38001026
:102A80003A000700002A3CD0AB789A18D2B204E092
:102A90000133DBB20E719A4233D04946C918087926
:102AA000FF28F5D05E464D46049F00236B7003E679
:102AB0005E46049FFDF76CFC50E65D465422002103
:102AC0002800FFF7B7F81022FF21281DFFF7B2F802
:102AD00028002022FF211430FFF7ACF8049BAB70D4
:102AE00064E65D46FAE7FFF7D1FB021E00D1E3E59D
:102AF000D37891781B020B4340460CA900F0E2F812
:102B0000EBE5330029003A00099800F017FC059B1B
:102B1000ED191B78B34200D37CE6C3E7FFF7B8FB9F
:102B2000021E00D1C8E5404613780CA900F0CAF88F
:102B3000D3E52189FDF744FC021EF4D1BCE5022A4D
:102B40000FD0FFF7A7FB021ED2D1B5E5FDF72CFC95
:102B5000021E00D1B0E5122340460CA900F0B2F8E5
:102B6000BBE5FDF729FC021EC2D1A5E5F8B5574625
:102B70004E46DE4645460C00E0B516001F00002A12
:102B80003CD01F4B00259A46702399461D4B9B460F
:102B900017E05B462000997800F092FB00281FD0D8
:102BA00021004046FFF75AFA002819D0A378DA0925
:102BB000012A1CD00A9A013513702378E418B54213
:102BC0001CDA6378052B0BD1E3789B079B0FBB4284
:102BD00006D153464A461B789846A3781A42D8D065
:102BE0000020F0BCBB46B246A946A046F8BD0B9AF1
:102BF000013513702378E418B542E2DB0120F0E7D9
:102C00001C100020881400200B007F2010B51840F5
:102C1000DB0934334000044AC018044B1168C01863
:102C200000F026FB10BDC046DC14002088140020F4
:102C300070B57F240F480C4064000419CD09641955
:102C400030342079C00701D5002070BD01262579D8
:102C50000948354300782571FFF78EFA0028F4D132
:102C60000122237993432371237903329343237100
:102C7000EAE7C046881400201C1000207F22054B84
:102C80000A405200C9099B185B1830331879C007F5
:102C9000C00F70478814002070B5094C0600082248
:102CA00020000D00FEF7CCFF00238021E360A3602D
:102CB0002B783000994300220023FFF7B9FF70BD45
:102CC000EC130020F8B5CE4647469046264E80B518
:102CD0008146082230000D001F00FEF7B1FF434679
:102CE000B3600023F381EC79AB7924021C43231CED
:102CF000BC4200D93B1C9FB2B381002C0ED0002FE8
:102D000018D04346002B2CD03B1C402F1BD89FB221
:102D100033787F2B1CD80021144A0FE080212B78B8
:102D20000022994348460023FFF782FFC0BCB94602
:102D3000B046F8BD7F230022317899433B004846D6
:102D4000FFF776FFF2E740239FB233787F2BE2D97B
:102D5000064C3A0041462000FEF772FF8021220017
:102D6000ECE70020E2E7C046EC130020AC130020A3
:102D700010B5142200210248FEF75CFF10BDC046CA
:102D8000EC130020014B18617047C046EC13002083
:102D900010B5054C010008222000FEF751FF00236A
:102DA000A360E36010BDC046EC13002070B5384C42
:102DB0001D0023780600DA09C9098A4210D00020D4
:102DC000002D00D070BD21003000FFF739F92369D4
:102DD000002B03D022000321300098470120F1E7A7
:102DE000A0687F2B05D8002834D02A002949FEF797
:102DF00027FFE289A1685219E38892B24919E2815A
:102E0000A160934214D03F2D12D9A389981A051CB2
:102E100080B240282AD82078ADB27F2828D8002157
:102E20009A4232D01B4A2B003000FFF701FFC9E75E
:102E30002369002B05D0220002213000984700288A
:102E40000AD0802123780022994330000023FFF725
:102E5000EFFEB7E70020B5E700213000FFF79EF94D
:102E600030008021FFF79AF90120ABE74025D2E737
:102E70009A4207D0074C2A002000FEF7E1FE80218D
:102E80002200D0E780210022CDE70022CBE7C04618
:102E9000EC130020AC1300207047C046012070479F
:102EA0007047C0467047C04642000C4B1218920053
:102EB00010B59B185C78FFF7EFF9002801D10020CE
:102EC00010BDFFF7F1F90028F9D1002CF7D021004F
:102ED000FFF7D4FE01235840C0B2F1E77014002080
:102EE000F8B50D0016001C00002801D00020F8BD28
:102EF000124F00207978FFF787FE0028F6D0002DCA
:102F00000ED1102CF2D80E4D220031002800FEF711
:102F100097FE23002A0079780020FFF789FEE6E774
:102F2000084805740F2CE1D811300500220031004B
:102F30000134FEF785FEA4B2013DEAE770140020DB
:102F4000501400204014002010B50C22002102482B
:102F5000FEF770FE10BDC0467014002001207047BF
:102F600010B50C2200210248FEF764FE10BDC046D9
:102F700070140020F0B54B7906000D0083B0032BD0
:102F80000AD10879C400241A1234A4B2944203D896
:102F9000194F7B78002B03D00024200003B0F0BD34
:102FA000097869184B78212BF6D1B9600B780200AB
:102FB000C9187B1C0193BB1C009330000323FFF74F
:102FC000D5FD0028E8D0AB79012B01D1EB79FB705E
:102FD0000123BB71AB78B9783B70BB68DA791B7A97
:102FE0001B021343BB800029D7D010233000034AB3
:102FF000FFF71EFED1E7C0467014002060140020C9
:103000001F23F0B514001278050083B01340012B84
:103010001BD1604E20793378984216D16023180076
:103020001040134208D020280FD163780B2B0CD806
:10303000594A9B00D3589F46012918D1E378A178BB
:1030400062781B020B43062A02D0002003B0F0BDB9
:103050001B0A212B00D181E0222BF6D10020FDF7A5
:10306000A7F921000200B3882800FFF72BFE0120FA
:10307000ECE70129FBD1E1780020F171FFF70EFFA9
:103080000028E2D021002800FFF706FE0120DDE73E
:1030900001296DD00329EAD1E079A3790002184310
:1030A000E278A178041C102800D910243B4BA4B26C
:1030B000002907D0012805D91878884202D1013C9F
:1030C000374BA4B200200094FDF76CF90120BDE756
:1030D0000129D7D00329CAD1A1780020B171FFF707
:1030E000DBFE0120B2E70129C1D1E379A0791B02FF
:1030F0000343E278A178181C102B00D9102080B26D
:10310000002943D0012B41D90126244F01383970C1
:1031100080B27B1C00900020FDF742F933189BB26F
:10312000002B00D191E73A0021002800FFF7CAFDEB
:1031300001208BE701299AD1012321002800194A97
:10314000FFF7C0FD012081E7012990D10123210073
:103150002800154AFFF7B6FD012077E7B268002A7C
:1031600000D172E7210028001378FFF7ABFD6DE76F
:10317000E379A2791B021343102B00D965E72100E4
:103180002800064AFFF79EFD01205FE7034F002657
:103190003B00BFE7701400204839001040140020A5
:1031A00041140020761400207714002070B51B4DC8
:1031B0000400A8786E7882B0884204D000208E4245
:1031C00015D002B070BD9BB2864211D0144E002AB9
:1031D00017D100930021330000200232FDF7E2F8FE
:1031E000102332002000A978FFF722FDE9E79BB207
:1031F000002A0CD100201A000A49FFF751FE0120D5
:10320000DFE7320002210020FFF74CFEE8E7002054
:103210000121044AFFF746FE0120D2E77014002086
:10322000601400205014002000B5030083B0002972
:1032300010D00020012B07D80A78002A04D00B48B0
:10324000C2540120012A01D003B000BD1800FFF7CD
:1032500033F8F9E7012301A900200B80FFF72CF8D0
:103260000028F1D00122014B1A70EDE77C140020F8
:10327000037870B5DB0704000E00DD0F002B17D1BB
:1032800003785B0701D5280070BD01213000494259
:1032900000F0C2F92378DB07DD0F002B0AD1237879
:1032A0005B0708D40422237801251343237002E02E
:1032B0000025E8E70025300000F08EF9E3E7C0467E
:1032C000437902791B021343C2785B0592075B0DB9
:1032D000920F022A1DD0032A0CD00020012A08D107
:1032E00002394A425141124A94466144994240414E
:1032F000C0B2704702394A1E91410E4A49421140FC
:103300008022D20094460020614499424041C0B2DC
:10331000EFE7022905D0002040229A424041C0B286
:10332000E7E7054A981843425841C0B2E1E7C04672
:10333000FF03000040FCFFFF00FEFFFF8A1870B58E
:10334000914207D27F264C78052C04D00C780919BD
:103350008A42F8D870BD34008D782C40640004197E
:10336000ED0963550C7809198A42ECD8F2E7C0469A
:1033700070B5040000690E00002803D00121494205
:1033800000F04AF925896089A288A9B283B28542F2
:103390002CD3CD1AADB2002D2ED0AA4208D2914224
:1033A00030D3891A8BB263819A4203D89B1A9BB29D
:1033B0009A42FBD9E28821685204520C53433000F0
:1033C000C918FEF73DFC63890125591C89B2A28802
:1033D0008B4213D900215200891A89B22069618178
:1033E000002801D000F0F8F8280070BD5500ED1A53
:1033F0004D19ADB2002DD0D1618989B252009142F0
:10340000ECDBE9E789188BB26381CDE7F8B50400FE
:10341000C0680E00002803D00121494200F0FCF8EA
:10342000258920896189A288ADB283B28FB2884292
:1034300029D3DB1B9BB29A4209D8E779FF0906D151
:10344000E068002801D000F0C7F83800F8BD9542C8
:103450001ED32B009B1A9BB29342FBD2E2882068BA
:103460005204520C53433100C018FEF7E9FB6B1CA9
:103470009BB2A2889D4218D9002352009B1A9BB28E
:1034800001272381DCE75100C91B5B189BB2D2E7FF
:103490002B00E28820685204520C53433100C018BC
:1034A000FEF7CEFB0135A288ABB252009342E7DBB8
:1034B000E4E7C04610B50400C068002803D001212D
:1034C000494200F0A9F82069002803D001214942AF
:1034D00000F0A2F80023E06863812381002801D076
:1034E00000F07AF82069002801D000F075F801207A
:1034F00010BDC04610B51920FCF7DCFFD023802298
:103500001B0692045A6210BD10B5024800F004F880
:1035100010BDC046101B002010B588B004000D225D
:1035200000216846FEF786FB0D22002104A8FEF765
:1035300081FB4B236A466846137004A90D2200F0F4
:1035400043F81521082220006944FEF779FB08B0F2
:1035500010BDC04610B583070AD00300032102E066
:1035600001330B4205D01A78002AF9D1181A10BD80
:10357000030019680C4A0D4C8A188A4322420FD165
:103580005968094A04338A188A43224208D1596883
:10359000054A04338A188A432242F1D000E00133FD
:1035A0001A78002AFBD1E1E7FFFEFEFE80808080D2
:1035B000F8B5C0460000000001B40248844601BCD2
:1035C000604700BF1502002001B40248844601BCD8
:1035D000604700BF090E002001B40248844601BCC8
:1035E000604700BFED01002001B40248844601BCE1
:1035F000604700BFD90E002001B40248844601BCD8
:10360000604700BFD90E002001B40248844601BCC7
:10361000604700BF110A002001B40248844601BC83
:10362000604700BF5D01002001B40248844601BC30
:10363000604700BFC100002001B40248844601BCBD
:10364000604700BFC90A002001B40248844601BC9B
:10365000604700BF790A002001B40248844601BCDB
:10366000604700BF390A0020011400102D1400101B
:1036700011160010251C0010911A0010951B001047
:103680003915001049140010691400107D14001041
:10369000BD09001085140010710D0010C913001031
:0C36A0006906001009350010B10200108E
:1036AC005250323034300000000000005353343993
:1036BC0045205765624849440000000031323334DC
:1036CC00353600000A2A2A2A2050414E4943202A26
:1036DC002A2A0A000A0000004E6F207370696E6C73
:1036EC006F636B732061726520617661696C6162D6
:1036FC006C650000486172647761726520616C6171
:10370C00726D20256420616C726561647920636C34
:10371C0061696D65640000004861726420617373B7
:10372C006572740052656C6561736500626F6F74CD
:10373C00325F77323571303830000000322E322E45
:10374C00300000007069636F00000000737334393F
:10375C00655F776562686964000000004A756E20D9
:10376C003232203230323600556E68616E646C65D0
:10377C00642049525120307825780A006570202544
:10378C003032582077617320616C726561647920E6
:10379C00617661696C61626C6500000043616E2743
:1037AC007420636F6E74696E75652078666572201F
:1037BC006F6E20696E616374697665206570202573
:1037CC00303258004C454400090400000902220024
:1037DC0001010080320904000001030000000921EE
:1037EC00110100012215000705810310000A0000D9
:1037FC000600FF0901A101150026FF0F75089502AF
:10380C0009028102C0000000120100020000004009
:10381C00FECA0040000101020301000006005250E4
:10382C00D3F075423037001006005250E182887F89
:10383C003837001006005250ABB3605348370010B5
:10384C0006005250BBFF3CB65037001006005250D9
:10385C00861C030258370010060052505422A29DB9
:10386C006837001005005250DE65F4680C490010F2
:10387C000D0A0000D823001040250010CA250010A6
:10388C00182500102A250010082500107824001097
:10389C002424001018240010E0280010C628001062
:1038AC00B826001000290010B8260010AE28001011
:1038BC009A280010B8260010862800109A270010AD
:1038CC00B82600104C2B00103E2B0010322B001091
:1038DC00B8260010B82600101C2B00103E2B001030
:1038EC00B8260010B8260010B8260010B826001014
:1038FC00B8260010B8260010B8260010E62A0010D2
:10390C009A0B00209A0B0020E40B0020040C0020E2
:10391C00420C0020540C0020900B002000000000F2
:10392C00492F00105D2F0010612F0010752F001013
:10393C0001300010AD310010000000004A300010C2
:10394C00E630001048310010343100104A300010BD
:10395C004A3000104A3000104A3000104A30001033
:10396C009030001072300010D0300010090052500E
:08397C0000000002D03700102A
:103984002838001034380010403800104C3800102B
:10399400583800106438001070380010783900105E
:1039A400F0B5C646150000B504001E000268EFF32A
:1039B400108172B61368002BFCD0BFF35F8F042311
:1039C400E356002B2DDB2268BFF35F8F00201060CD
:1039D40081F31088D0221206127852B290469A428D
:1039E40003D1002080BCB846F0BD00270BE023685B
:1039F400BFF35F8F1F6081F310882800310000F04F
:103A0400FFFE0028EDD12268EFF3108172B613682F
:103A1400002BFCD0BFF35F8F23797F2BE7D943467C
:103A240002E0D0231B061B6823712368BFF35F8F5A
:103A340000221A6081F310880120D3E7F0B5C6464E
:103A440000B50D00040000F0C3FEFA2206000F00CA
:103A5400002328000021920000F0B2FE80233618D3
:103A64004F411B069F4202D30126174F7642D023B3
:103A74001B061B68002598460BE02368BFF35F8F85
:103A84001D6081F310883000390000F0B9FE002871
:103A940018D12268EFF3108172B61368002BFCD0A2
:103AA400BFF35F8F23797F2BE7D9434623712368C4
:103AB400BFF35F8F00221A6081F31088012080BC5D
:103AC400B846F0BD0020FAE7FFFFFF7F0268EFF37E
:103AD400108172B61368002BFCD0BFF35F8FFF23F5
:103AE40003710368BFF35F8F00221A6081F31088AB
:103AF40040BF70470022154B10B59A60DA601A6116
:103B04005A619A61DA611A625A629A62DA621A63D3
:103B14005A639A63DA631A645A649A64DA641A65B3
:103B24005A659A65DA651A665A669A66DA661A6793
:103B34005A679A67DA67F03292000021044800F06D
:103B44004FFE044B044A1A6010BDC04600001050DA
:103B540020170020E41A002080011050F0B54E46D2
:103B64004546DE465746E0B5214B00249E6D0125AF
:103B740085B0002E22D01F4B9A46012399461E4B36
:103B8400984601E0202C19D02A00230001342F008C
:103B94003240E4B26D00002AF4D0524697654A469A
:103BA4005B085B0022409B185B01434418009B4662
:103BB40000F030FC002808D1BE43E3D105B0F0BCCE
:103BC400BB46B246A946A046F0BD5B46E0219A78C2
:103BD400DB8A01A883600023C900018001210271EE
:103BE400437100F037FC584600F0B0FBE4E7C046F0
:103BF4000000115000301150E01600209823F0B559
:103C0400C646C64A00B5D55880232E009B02102410
:103C140084B01E401D4273D0C14BC24C9A6AC24B41
:103C240000261A603B23E35C022B00D1F4E07B23E3
:103C3400E35C022B00D10CE1BB23E35C022B00D13B
:103C4400FBE0FB23E35C022B00D135E13C23FF3393
:103C5400E35C022B00D122E17C23FF33E35C022BE3
:103C640000D10FE1BC23FF33E35C022B00D1FCE065
:103C7400FC23FF33E35C022B00D1A6E1AB4BE35CF6
:103C8400022B00D196E1AA4BE35C022B00D185E123
:103C9400A84BE35C022B00D174E1A74BE35C022B3D
:103CA40000D163E1A54BE35C022B00D12AE1A44BD4
:103CB400E35C022B00D10BE1A24BE35C022B00D1AD
:103CC4008FE1A14BE35C022B00D1A6E1002E08D1C9
:103CD4009E4B1B78002B04D180219D4A903389028E
:103CE400D150C0228D4B01A89B6C92005B055B0DEB
:103CF400012180260280436000F0ACFB954CB602A3
:103D0400EB0600D57CE080235B021D4232D01E43CB
:103D1400012302249846834FBB7E002B14D000F06D
:103D240077FD012800D96FE0C022002138009201FC
:103D340000F012FB380000F009FB00F069FD0128D7
:103D440002D9834B5C661C664346FB702037012C0A
:103D540001D00124E0E7C02301A8DB007E4A0380F0
:103D640002AB12CA12C3012100F074FB8022784B0B
:103D740092021A6580235B011D420ED18023DB0170
:103D84001D4221D180231B021D422CD1AE4200D002
:103D9400C0E104B080BCB846F0BD00241E435F4BB4
:103DA4001C60FFF7A7FE80236A465B0093801472B1
:103DB400012101A800F04EFB8022654B12031A6515
:103DC4008023DB011D42DDD01E43802301A8DB00DC
:103DD4000380012100F03EFB10225D4B1A65802315
:103DE4001B021D42D2D01E43A02301A8DB00038086
:103DF400012100F02FFB8022554B12011A65C5E703
:103E0400FFF7ACFE26007EE7544B444A1C66536E13
:103E14002340A342FBD187E73833E65C002E00D170
:103E240005E70233E25C002A00D100E7200000220B
:103E34002030E25400F0B8FAF9E6B833E75C002F1A
:103E440000D1FEE60233E25C002A00D022E13E000B
:103E5400F7E67833E75C002F00D1EDE60233E25C4D
:103E6400002A00D00EE13E00E6E6B933FF33E75CFA
:103E7400002F00D1FCE60233E25C002A00D0F8E017
:103E84003E00F5E67933FF33E75C002F00D1E9E625
:103E94000233E25C002A00D0E2E03E00E2E639337D
:103EA400FF33E75C002F00D1D6E60233E25C002A40
:103EB40000D0CCE03E00CFE6F833E75C002F00D121
:103EC400C4E60233E25C002A00D0B8E03E00BDE65E
:103ED400234BE75C002F00D1EEE60233E25C002ABC
:103EE40000D010E1174BE35C022B00D18BE0164BA2
:103EF400E35C022B00D0F4E61A4BE35C002B00D009
:103F040090E0EEE6184BE75C002F00D1CFE60233D9
:103F1400E25C002A00D0EEE03E00C8E6000011504A
:103F240000400540E0160020D81600203B020000A7
:103F34007B020000BB020000FB0200003B03000008
:103F44007B030000BB030000FB030000211B0020D7
:103F540000301150100002000000105000201150D9
:103F64007A030000FA0300003A0300006C4BE75C9C
:103F7400002F00D196E60233E25C002A00D0B2E0C2
:103F84003E008FE6674BE75C002F00D185E60233E5
:103F9400E25C002A00D09EE03E007EE6624BE75CD5
:103FA400002F00D174E60233E25C002A00D08AE0DC
:103FB4003E006DE65D4BE75C002F00D163E6023303
:103FC400E25C002A77D13E005DE6F933FF33E75C1B
:103FD400002F00D152E60233E25C002A62D13E0097
:103FE4004CE6534BE35C002B00D16AE6EF239B00C5
:103FF400E25C002A00D17AE70022E2541C3BE0187C
:1040040000F0D2F973E74A4BE35C002BEED1494B45
:10401400E35C022B00D064E63E00474BE35C002BDC
:1040240000D153E6FF239B00E25C002A00D158E64E
:104034000022E2541C3BE01800F0B6F951E62000DF
:104044000022E030E2543E0000F0AEF9FEE520002C
:1040540000222130FF30E2543E0000F0A5F9FBE5D8
:10406400200000226130FF30E2543E0000F09CF951
:10407400F8E520000022A130FF30E2543E0000F0B9
:1040840093F9F5E5200000226030E2543E0000F090
:104094008BF9D1E520000022A030E2543E0000F06C
:1040A40083F9CEE520000022E130FF30E2543E00E7
:1040B40000F07AF9E2E50022E2541C3BE01800F03B
:1040C40073F93E00DFE50022E2541C3BE01800F0E7
:1040D4006BF93E00DCE50022E2541C3BE01800F0E2
:1040E40063F93E00D9E50022E2541C3BE01800F0DD
:1040F4005BF93E00D6E50022E2541C3BE01800F0D8
:1041040053F93E00D3E50022E2541C3BE01800F0D2
:104114004BF9E7E631000948694000F089FBC046E5
:10412400FA020000BA0200007A0200003A0200001B
:10413400BA030000FB030000FA0300007437001008
:10414400F0B5D6464F464646C0B50200838A008B7A
:104154008A46041C984200D91C1CD5788026280065
:10416400471EB841A4B2F60026434003304301265B
:1041740075401B1BD57055789BB29382002D37D1A7
:104184005146D6688D01611E761988461569002C42
:1041940029D006293AD933002B439B0736D16B1C0F
:1041A400F31A022B32D9231F9B0801339C460027A4
:1041B4000023E9580137F1500433BC45F9D863466C
:1041C40041469B00ED18F618CF1A9C4209D02B7873
:1041D4003370002F05D06B787370012F01D0AB784A
:1041E400B3701569938A2D19156180221202104348
:1041F400002B02D18023DB0118435346002B00D04F
:104204000004E0BCBA46B146A846F0BD0023EF5C0A
:10421400F75401339C42FAD11569938AE3E7C04607
:104224008368F0B51B680500002900D01B0C9B05B2
:10423400980D6B78002B08D1EB8AC318EB822B8B7B
:10424400834201D90023AB82F0BDEB688901461E8D
:10425400B4462A695C18002827D0062E2BD90131D0
:104264005B18D31A022B26D9130023439B0722D1B0
:1042740000230021061FB6080136E7580131D75044
:1042840004338E42F9D86346B600A41992199F1BD1
:10429400B04209D023781370002F05D0637853708F
:1042A400012F01D0A37893702A69EB8A1218C318DE
:1042B400EB822A61C3E70023E15CD15401339842C5
:1042C400FAD12A69F1E7C04610B5040083680021D9
:1042D4001B68FFF7A5FF63681B685B0002D5238B8F
:1042E400834200D010BD01212000FFF799FFF9E7B8
:1042F400084A0300126C0020920703D49A78D2096A
:10430400012A00D07047D87E023843425841C0B2D7
:10431400F8E7C0460000115010B5FFF7E9FF002888
:104324000CD00749074B8C46074A9B6A12686344C2
:104334009B1A0020C6229A424041C0B210BDC0461A
:10434400E0FCFFFF00400540D816002000238376E0
:10435400436103617047C04610B58368002901D0EA
:104364001C682140002A12D08024E4001143224218
:104374000DD01A6822420CD1084A0A401A60084A31
:10438400126C920703D40C23033BFDD2836819609B
:1043940010BD8178034800F04BFAC046FFFBFFFFD5
:1043A4000000115088370010436870B50021802543
:1043B4001E680400FFF7C4FE134B6D011B6C05431C
:1043C4009B070FD5A3785B060FD0104B1E408023AC
:1043D4009B05334362680021136020002A00FFF725
:1043E400BBFF70BDA378DB09EFD0A38A002BECD010
:1043F40001212000FFF7A4FEA023054ADB0532407B
:1044040005431343E6E7C04600001150FFFFFFAF2A
:10441400FFFFFFDF70B5857E0400002D14D0FFF789
:1044240053FFA38A002B01D1280070BD2000FFF7A1
:1044340073FF002803D0012300252377F4E720002D
:10444400FFF7B2FF0025EFE78178014800F0F0F9AB
:10445400A8370010F0B5CE46474680B5437805002E
:104464000E0085B0062B08D86B4A9B00D3589F4694
:104474006A4A13780133DBB21370694B1C686269B2
:10448400EFF3108172B61368002BFCD0BFF35F8F7B
:10449400A1612000290000F0ABF96269A369BFF3B0
:1044A4005F8F0021116083F31088002804D105B0C8
:1044B400C0BCB946B046F0BD32006978287800F037
:1044C400AFF9F4E70121574B1A788A431A701A7826
:1044D40001318A431A7000225A701A7802318A43D1
:1044E4001A70CAE7504B514F9946514B00249846D5
:1044F4003A7810E043461B6861015B18002B06D034
:10450400DB69002B03D06968287898473A7801342E
:10451400E4B2944217D8A242ECD8A31A5B014B44EC
:10452400EEE7404B1A78D207C1D504211A780A4322
:104534001A70A2E73B4B1A78D207B8D504211A782F
:104544008A431A7099E7374F3B785B072BD50422CF
:104554003B78002193433B706B460632981D00F074
:104564003FF92B7801AC2370052363702C4B1B6837
:1045740098465A69EFF3108172B61368002BFCD089
:10458400BFF35F8F434640469961210000F030F944
:1045940043465A699B69BFF35F8F0021116083F31F
:1045A4001088002831D1FB78DB0700D47FE76B4605
:1045B4000A220021981D00F013F92B7801AC237016
:1045C400032363706B686360154B1D686A69EFF3BE
:1045D400108172B61368002BFCD0BFF35F8FA96102
:1045E4002800210000F004F96A69AB69BFF35F8F0A
:1045F4000021116083F31088002800D157E73200AE
:104604006178207800F00CF951E732006178207865
:1046140000F006F9C7E7C0460C390010221B002041
:10462400E01400208814002028390010201B0020EA
:10463400A813002010B5084C2378002B0AD180233E
:10464400064807495B051A68C25004338B42FAD105
:104654000123237010BDC046231B0020A4150010A5
:104664000001001010B5014B984710BDA51500209E
:10467400064B5A6802609A684260DA6882601A6976
:10468400C2605A6902619B6943617047000002403D
:104694000268064B5A6042689A608268DA60C268AF
:1046A4001A6102695A6142699A61704700000240C6
:1046B400034B1A68C0239B009343024A136070475C
:1046C4000C8001400C900140054B1A6880239B002C
:1046D4005340C02292001340024A13607047C04600
:1046E4000C8001400C9001401423F0B5D6464F468F
:1046F40046469A46C0B581461888043386B0984623
:104704000E001B882949140098475346070018884F
:10471400434627491B889847534605001888434653
:1047240024491B8898478046FFF784FF6846FFF7B3
:104734009FFFB847A847FFF7C7FF221E20D0C0211C
:1047440008270220490511E0002C14D0131B0D2B5F
:1047540024D9002D0AD02300002A05D00B6E013A7B
:104764003370130001362343002B09D03D008B6ABC
:104774001D401842E8D1002DEDD123001343F5D19B
:10478400FFF796FFC047FFF76DFF6846FFF780FF0E
:1047940006B0E0BCBA46B146A846F0BD4B461B780D
:1047A400013C0B6601239C46E144E4E749460000D2
:1047B40045580000464300007047C0460000000012
:1047C40001B40248844601BC604700BF611B00106D
:1047D40001B40248844601BC604700BF8D1000103C
:1047E40001B40248844601BC604700BF351C001078
:1047F40001B40248844601BC604700BF0D34001078
:1048040001B40248844601BC604700BF710F001028
:1048140001B40248844601BC604700BFF50400109F
:1048240001B40248844601BC604700BF85220010E1
:1048340001B40248844601BC604700BF0105001072
:10484400D4370010AC360010B8360010C83600104B
:104854001000000000000000000001000000000043
:104864000000000000000200000000000000000042
:104874000000030000000000000000000000FF0032
:104884000000000001B5486801318E4600477046BB
:1048940009380149884701BDF908001000000000EB
:1048A4000000000000000000000000000000000004
:1048B400281000200000000000000000000000009C
:1048C400503300004C3300005433000052330000D6
:1048D4004D5300004D4300005334000043340000A6
:1048E400E414002010000C00000000000000000090
:1048F400000000000000000000000000FF000000B5
:084904000000000000000000AB
:04000005100001E9FD
:00000001FF
